:020000020000FC
:10000000DAC018951895189518951895189509C07F
:100010001895189518951895189518951895189578
:1000200018952FB60F930CEF02BF0FE16017B9F4CC
:10003000662794980FEF802E0CE35394501651F4DA
:1000400055244394401631F44424339408E1301687
:1000500009F433240FEF02BF0F912FBE18954030E3
:1000600089F426E0949800000000949A0000959A84
:100070000000979A0FEF05BB96980000969A64D0FF
:1000800095983FC0413049F42CE0979A0FEF05BB9B
:1000900096980000969A58D034C0423049F425E131
:1000A000979A0FEF05BB96980000969A4DD029C0FD
:1000B000433049F42EE1979A0FEF05BB9698000064
:1000C000969A42D01EC0443049F427E2979A0FEF27
:1000D00005BB96980000969A37D013C0453049F476
:1000E00020E3979A0FEF05BB96980000969A2CD0C4
:1000F00008C029E3979A0FEF05BB96980000969ADF
:1001000023D0439507E0401751F44427639402E15C
:10011000601629F466246395B3950FEF702E411590
:1001200081F40091E200889483990894001F009361
:10013000E2000091E300889482990894001F0093E4
:10014000E3000F912FBE1895D0E0C5EEC60DD11D6E
:100150009880D0E0C0E6C20FD11D3FEF68940991AE
:10016000092109F0377F0991092109F03B7F0991A5
:10017000092109F03D7F293311F4D0E0C0E609914F
:10018000092109F03E7F0991092109F0E8940991BC
:10019000092109F03F770991092109F03F7B099175
:1001A000092109F03F7D0991092109F03F7E0EF0F8
:1001B000979835BB0895F894479A0CEF02BF04E076
:1001C00003BF02E009BF02E00EBF0FE50DBF0FEF56
:1001D0000ABB00E00BBB0FEF07BB03E108BB0FEF4F
:1001E00004BB0FEF05BB00EF01BB0CEA02BB0FEF36
:1001F00006B900E007B900E00BB906E800BD00E071
:1002000000BD0CE009B994989598969A112433246E
:1002100044245524662766244427772488244427C9
:100220005527AA2779E000E0F02EEE24DD24882768
:1002300096E0BB2710928701109284010E94790DED
:10024000ADD70E94440E789483997EC082992BC0CA
:1002500083997AC0829978C0052D033009F0F8CFD0
:10026000AEE1E0E6F0E001E0019300E00193AA9541
:10027000D1F70AEA0BBB05E508BB0FEF8016E9F7DB
:100280008824AEE1E0E6F0E000E0019301E00193B4
:10029000AA95D1F705E50BBB0AEA08BB0FEF80165C
:1002A000E9F78824DDCFECE9F0E000E2019300E219
:1002B000019300E201930EE301930CE4019309E63C
:1002C00001930EE601930BE601930EE201930EE219
:1002D000019300E2019300E2019300E2019300E246
:1002E000019300E2019300E2019300E2019300E236
:1002F000019300E012E100938101109382017727BE
:10030000FF2408E10AB90000000000000CE40E948C
:10031000190C09E60E94190C0EE60E94190C0BE656
:100320000E94190C0E941D0C0FEF801611F48824F6
:100330001ED00FEF7016B1F77724DFD79A9511F41E
:1003400096E052D71DD0EECF0FEF801611F488241F
:100350000ED00FEF7016C1F77724CFD79A9519F406
:1003600096E00E94F408F7D7E5D70AD0EDCF1F2D0D
:10037000113011F4BAD60895123009F4D9D608957F
:10038000072F0F77013021F477FF25D40BD428C035
:10039000023021F477FFDCD42BD422C0033021F4C7
:1003A00077FFFED36BD11CC0043021F477FF78D0E7
:1003B0002CD016C0053021F477FF5ED105D110C0D6
:1003C000063021F477FF41D5CDD40AC0073021F49F
:1003D00077FFF8D0A6D004C0093011F403D000C0D4
:1003E00070680895DFD3009181010A3309F0089500
:1003F00001E0F02E01E0702F0895002703D01A9538
:10040000E1F708950A95F1F70895052D0A3308F0EC
:1004100088C0003041F1AA2715E0011B10F0A10FA0
:10042000FCCF010F0130D9F5E7EFF0E0E60FF11D49
:100430001081E0E6F0E0EA0FF11D118312831383CF
:1004400014831583613059F5A03049F1E450F10966
:1004500001E0008301E0018301E0028301E0038306
:1004600001E004831CC06530D1F4E0E6F0E001E077
:10047000008301E0058301E0028701E0078701E0D6
:10048000048B01E0018F01E0068F01E003A301E08E
:1004900000A701E005A701E002AB01E007AB08956A
:1004A00059D4052D0A33E0F5E0E6F0E001E00083E1
:1004B00001E0058301E0028701E0078701E0048B8A
:1004C00001E0018F01E0068F01E003A301E000A736
:1004D00001E005A701E002AB01E007AB052D01300B
:1004E000F8F00A95AA2715E0011B10F0A395FCCFA0
:1004F000010FA3951A2F110F110F1A0FE0E6F0E06C
:10050000E10FF11DE450F10901E0008301E00183F6
:1005100001E0028301E0038301E00483AA9551F71F
:100520000895162F052D079510F40FE1100F1030C8
:1005300069F0113081F01230A9F01B33E0F01B3369
:1005400049F11C3391F11D33B9F13BC0E0E6F0E015
:1005500000E8008336C0E0E6F0E000E1008300E858
:1005600001832FC0E0E6F0E002E0008300E10183B8
:1005700000E8028326C0E0E6F0E0E10FF11DE35061
:10058000F10900E0008302E0018300E1028300E85A
:10059000038317C0E0E6F0E000E000AF00E001AF49
:1005A00004E002AF00E803AF0CC0E0E6F0E000E0DA
:1005B00002AF04E003AF05C0E0E6F0E000E003AF07
:1005C00000C00895C7D30895062F0130A9F4052D62
:1005D0000B3090F00A3380F4E0E6F0E00CE3E00F3B
:1005E000F11D10916000029100936000AAE3029156
:1005F0000183AA95E1F71083052D0030E1F10B305E
:1006000030F0033370F00A3308F08BCF34C0A52CE0
:10061000AA0C0A2DAA0CA00E0CE3A01608F0A01A32
:1006200020C0152D0AE0AA27101B10F0A395FCCFBF
:10063000100FAA24AA950A2F000F000F000F0A0F0F
:10064000A00E012F010F010F010F010F010F010F6C
:10065000A00EAA94103009F4A3940CE3A01608F09D
:10066000A01AE7EFF0E0E60FF11D1081E0E6F0E000
:10067000EA0DF11D108308956DD3089510E0052D46
:10068000079508F41FE1EAE4F3E0E10FF11DE60F3E
:10069000F11D09943EC042C046C04AC04EC054C07D
:1006A0005AC060C068C070C07AC082C08CC096C09A
:1006B000A0C0ACC0BAC0C8C0D4C0DEC0E8C0F2C0E0
:1006C000FAC004C10CC116C11EC126C12EC136C15B
:1006D0003CC142C146C14AC14EC152C158C15EC1AE
:1006E00064C16CC174C17EC186C190C19AC1A4C1EC
:1006F000B0C1BEC1CCC1D8C1E2C1ECC1F6C1FEC11E
:1007000008C210C21AC222C22AC232C23AC240C2AF
:100710000000E0E6F0E000E801A741C2E0E6F0E01A
:1007200000E801A73CC2E0E6F0E000E801A737C21C
:10073000E0E6F0E000E801A732C2E0E6F0E000E128
:1007400001A700E800A72BC2E0E6F0E004E001A763
:1007500000E800A724C2E0E6F0E002E001A700E81C
:1007600000A71DC2E0E6F0E001E001A700E100A75C
:1007700000E807A314C2E0E6F0E001E001A704E00E
:1007800000A700E807A30BC2E0E6F0E000E001A745
:1007900002E000A700E107A300E806A300C2E0E62C
:1007A000F0E001E000A704E007A300E806A3F7C11A
:1007B000E0E6F0E000E000A701E007A304E006A304
:1007C00000E805A3ECC1E0E6F0E000E007A301E0EB
:1007D00006A304E005A300E804A3E1C1E0E6F0E01D
:1007E00000E006A301E005A304E004A300E803A3DE
:1007F000D6C1E0E6F0E000E005A300E004A301E0DC
:1008000003A304E002A300E801A3C9C1E0E6F0E00D
:1008100000E003A300E002A300E001A301E000A3C5
:1008200004E0078F00E8068FBAC1E0E6F0E000E0E0
:1008300000A300E0078F00E0068F01E0058F04E0D1
:10084000048F00E8038FABC1E0E6F0E000E0058F25
:1008500000E0048F01E0038F04E0028F00E8018FC5
:100860009EC1E0E6F0E000E0038F01E0028F04E0CB
:10087000018F00E8008F93C1E0E6F0E000E0028F16
:1008800001E0018F04E0008F00E8078B88C1E0E6FB
:10089000F0E000E0018F02E0008F00E1078B00E84C
:1008A000068B7DC1E0E6F0E001E0008F04E0078BFD
:1008B00000E8068B74C1E0E6F0E000E0008F02E0A3
:1008C000078B00E1068B00E8058B69C1E0E6F0E0EC
:1008D00001E0078B04E0068B00E8058B60C1E0E6D1
:1008E000F0E000E0078B02E0068B00E1058B00E8FA
:1008F000048B55C1E0E6F0E001E0068B04E0058BD7
:1009000000E8048B4CC1E0E6F0E000E0068B02E07A
:10091000058B00E8048B43C1E0E6F0E001E0058BC5
:1009200004E0048B00E8038B3AC1E0E6F0E000E06D
:10093000058B02E0048B00E8038B31C1E0E6F0E0B8
:1009400001E0048B00E8038B2AC1E0E6F0E000E060
:10095000048B00E8038B23C1E0E6F0E000E8038BA2
:100960001EC1E0E6F0E000E8038B19C1E0E6F0E02C
:1009700000E8038B14C1E0E6F0E000E8038B0FC150
:10098000E0E6F0E000E1038B00E8048B08C1E0E65C
:10099000F0E004E0038B00E8048B01C1E0E6F0E046
:1009A00002E0038B00E8048BFAC0E0E6F0E001E02F
:1009B000038B00E1048B00E8058BF1C0E0E6F0E07A
:1009C00001E0038B04E0048B00E8058BE8C0E0E65F
:1009D000F0E000E0038B02E0048B00E1058B00E80F
:1009E000068BDDC0E0E6F0E001E0048B04E0058B5F
:1009F00000E8068BD4C0E0E6F0E000E0048B01E004
:100A0000058B04E0068B00E8078BC9C0E0E6F0E048
:100A100000E0058B01E0068B04E0078B00E8008F07
:100A2000BEC0E0E6F0E000E0068B01E0078B04E0EA
:100A3000008F00E8018FB3C0E0E6F0E000E0078B34
:100A400000E0008F01E0018F04E0028F00E8038FD7
:100A5000A6C0E0E6F0E000E0018F00E0028F00E0D9
:100A6000038F01E0048F04E0058F00E8068F97C034
:100A7000E0E6F0E000E0048F00E0058F00E0068F84
:100A800001E0078F04E000A300E801A388C0E0E6CE
:100A9000F0E000E0078F00E000A301E001A304E024
:100AA00002A300E803A37BC0E0E6F0E000E001A3BE
:100AB00001E002A304E003A300E804A370C0E0E6A1
:100AC000F0E000E002A301E003A304E004A300E8D7
:100AD00005A365C0E0E6F0E000E003A302E004A3A4
:100AE00000E105A300E806A35AC0E0E6F0E001E05B
:100AF00004A304E005A300E806A351C0E0E6F0E08B
:100B000000E004A302E005A300E106A300E807A3B8
:100B100046C0E0E6F0E001E005A304E006A300E83B
:100B200007A33DC0E0E6F0E000E005A302E006A375
:100B300000E107A300E800A732C0E0E6F0E001E032
:100B400006A304E007A300E800A729C0E0E6F0E060
:100B500000E006A302E007A300E800A720C0E0E64B
:100B6000F0E001E007A304E000A700E801A717C038
:100B7000E0E6F0E000E007A302E000A700E801A73C
:100B80000EC0E0E6F0E001E000A700E801A707C022
:100B9000E0E6F0E000E000A700E801A700C008954B
:100BA000D9D00895052D003051F0E7EFF0E0E60FC1
:100BB000F11D1081E0E6F0E0E00F11930895E7E108
:100BC000F1E0E60FF11D1081ACE3E0E6F0E01193F7
:100BD000AA95E9F70895BED0A52DA23040F0E0E631
:100BE000F0E0E395AA9501E00193AA95E9F708954D
:100BF000EDEFF5E0E60FF11D09941EC01DC01CC00D
:100C00001BC01AC019C018C018C01FC01EC01EC00B
:100C100037C036C035C034C034C03BC03AC039C01C
:100C200038C038C051C050C050C057C056C055C061
:100C300054C053C052C052C071C071D0E0E6F0E061
:100C4000EC0DF11D00E4008369C068C068D0E0E6E7
:100C5000F0E0EA0DF11D02E00083E0E6F0E0EB0DCC
:100C6000F11D00E10083E0E6F0E0ED0DF11D08E08C
:100C70000083E0E6F0E0EE0DF11D01E000834EC0E0
:100C80004DC04DD0E0E6F0E0EC0DF11D00E8008332
:100C900045C044C044D0E0E6F0E0EA0DF11D01E0BB
:100CA0000083E0E6F0E0EB0DF11D08E00083E0E6F4
:100CB000F0E0ED0DF11D00E10083E0E6F0E0EE0D67
:100CC000F11D02E000832AC029C029D0E0E6F0E04F
:100CD000EC0DF11D00E4008321C020C020D0E0E62F
:100CE000F0E0EA0DF11D00E00083E0E6F0E0EB0D3E
:100CF000F11D04E00083E0E6F0E0ED0DF11D00E2FF
:100D00000083E0E6F0E0EE0DF11D04E00083E0E694
:100D1000F0E0EC0DF11D00E2008300C00895052D08
:100D2000ACE3C52C0A950C3308F00A0FB02E0A95D7
:100D30000C3308F00A0FA02E052D03950C3308F094
:100D40000A1BD02E03950C3308F00A1BE02E0895E1
:100D500001D00895ACE3E0E6F0E000E00193AA954D
:100D6000E9F70895052D003009F46EC0013009F44B
:100D700010C00E3108F414C00E3109F431C00F3127
:100D800009F435C00B3308F43DC00B3309F455C0EA
:100D90005BC01CE297D01DE295D01EE293D054C0F8
:100DA0001DE215198FD01DE2150D1C3308F01C53E0
:100DB00089D01DE215191395CED01DE2150D1A9597
:100DC0001C3308F01C53C7D0052D023019F00D312B
:100DD00021F03AC01DE2BFD037C01FE073D034C04D
:100DE0001EE0B9D01FE0B7D010E1B5D02DC01CE295
:100DF000F0D01DE2EED01EE2ECD01BE2CBD01FE221
:100E0000C9D022C01AE41519C5D010E1150D1C3344
:100E100008F01C53BFD01AE4151913950CD110E13A
:100E2000150D1A951C3308F01C5305D1052D0A33F6
:100E300009F00AC01FE0AED007C01EE0FCD01FE0E2
:100E4000FAD010E1F8D000C0089584DF052D0330FA
:100E500008F437C00F3110F0A1F01BC00FE20519E4
:100E6000A52DAA0FA350E0E6F0E0E00FF11D10E879
:100E70001193AA9529F0EC39D9F7E0E6F0E0F8CF24
:100E800020C0E0E6F0E0ACE310E81193AA95E9F7A2
:100E900018C00FE0050D0C3308F00C53152D10523F
:100EA000110FA9E3A11BE0E6F0E0E00FF11D10E84F
:100EB0001193AA9529F0EC39D9F7E0E6F0E0F8CFE4
:100EC00000C00895062F073110F4A0E001C0A1E092
:100ED000E0E6F0E0E10FF11DA0830895062F0C304D
:100EE00010F4A1E005C0063110F4A2E001C0A4E0B6
:100EF000EFCF062F073010F4A0E009C0003110F446
:100F0000A1E005C0083110F4A2E001C0A4E0E0CFE8
:100F1000062F023010F4A0E01DC0073010F4A1E04D
:100F200019C00C3010F4A2E015C0003110F4A4E098
:100F300011C0033110F4A8E00DC0063110F4A0E197
:100F400009C0093110F4A0E205C00C3110F4A0E48E
:100F500001C0A0E8BDCF062F053010F4A1E019C0F4
:100F60000A3010F4A2E015C00E3010F4A4E011C055
:100F7000023110F4A8E00DC0063110F4A0E109C060
:100F8000093110F4A0E205C00C3110F4A0E401C056
:100F9000A0E89ECF062F033010F4A0E819C0063059
:100FA00010F4A0E415C0093010F4A0E211C00D3017
:100FB00010F4A0E10DC0013110F4A8E009C0053122
:100FC00010F4A4E005C00A3110F4A2E001C0A1E0D1
:100FD0007FCF062F033010F4A0E81DC0063010F4B8
:100FE000A0E419C0093010F4A0E215C00C3010F4D0
:100FF000A0E111C00F3010F4A8E00DC0033110F4CF
:10100000A4E009C0083110F4A2E005C00D3110F4CD
:10101000A1E001C0A0E05CCF062F073010F4A4E0EF
:1010200009C00F3010F4A2E005C0083110F4A1E0AF
:1010300001C0A0E04DCF062F083010F4A1E001C0A0
:10104000A0E046CF062F063010F4A4E011C00C300B
:1010500010F4A8E00DC0013110F4A0E109C0053181
:1010600010F4A0E205C0093110F4A0E401C0A0E82A
:101070002FCF062F063010F4A0E811C00A3010F46C
:10108000A0E40DC00E3010F4A0E209C0033110F44A
:10109000A0E105C0093110F4A8E001C0A4E018CF18
:1010A000ECE9F0E01091850171D000E3A00F100F82
:1010B000A19311930AE301931091860167D000E395
:1010C000A00F100FA19311930EE2019310E05ED0D8
:1010D00000E3A00F100FA193119300E018E000931C
:1010E00081011093820180D00895ECE9F0E0132D86
:1010F0004DD000E3A00F100FA19311930AE30193C9
:10110000142D44D000E3A00F100FA19311930EE211
:101110000193152D3BD000E3A00F100FA193119365
:1011200000E018E000938101109382015DD00895E2
:10113000ECE9F0E000E20193132D103011F41CE013
:1011400003C01D3008F01C5021D000E3A00F100F89
:10115000A03319F400E2019301C0A19311930AE3B3
:101160000193142D13D000E3A00F100FA19311933E
:1011700000E2019300E2019300E2019300E018E035
:1011800000938101109382012FD00895AA270AE0CD
:10119000101718F0101BA395FBCF08951092810132
:1011A0001092820110928301C09800000000C09A42
:1011B000002728D908E80BBB03E908BBC498000046
:1011C000C49A00271FD9089508E00BBB03E908BBA8
:1011D000C4980000C49A089500E00BBB03E908BB63
:1011E000C4980000C49A0895009181011091820171
:1011F0001850101B08F40895ECE9F0E0E00FF11D21
:1012000003950093810101910BBB03ED08BBC498CA
:101210000000C49A01910BBB07ED08BBC498000005
:10122000C49A01910BBB0BED08BBC4980000C49A93
:1012300001910BBB0FED08BBC4980000C49A01914B
:101240000BBB03EF08BBC4980000C49A01910BBB11
:1012500007EF08BBC4980000C49A01910BBB0BEFC9
:1012600008BBC4980000C49A01910BBB0FEF08BBE8
:10127000C4980000C49A00918101039500938101F4
:101280000895119100E01F70010F0BBB03E108BB33
:10129000C4980000C49A11911BBB03E508BBC49815
:1012A0000000C49A11911BBB07E508BBC49800005D
:1012B000C49A11911BBB0BE508BBC4980000C49AEB
:1012C00011911BBB0FE508BBC4980000C49A119193
:1012D0001BBB03E708BBC4980000C49A11911BBB59
:1012E00007E708BBC4980000C49A11911BBB0BE729
:1012F00008BBC4980000C49A08950091E300003030
:1013000011F450FF59600091E3000F3F21F450FFAA
:1013100002C05E7F54600091E200003011F451FF82
:1013200052620091E2000F3F21F451FF02C05D7F45
:101330005061089553FF0EC0577F7F7773957830C3
:1013400048F071E001E0F01619F402E0F02E02C05E
:1013500001E0F02E089555FF07C05F7D839587302B
:1013600019F4882701E0F02EE9EBF9E0E80FF11D10
:10137000099447C21DC048C04CC077C09CC0C7C0BC
:1013800040C23FC23EC23DC2ADC1B4C1C8C1E7C147
:1013900002C221C236C235C234C233C26CC087C059
:1013A00030C22FC22EC2B9C099C12BC22AC229C2D3
:1013B000ECE9F0E000E2019300E2019300E2019326
:1013C00000E2019300E2019300E2019300E2019345
:1013D0000EE3019304E5019309E601930DE6019301
:1013E00005E6019303E5019305E6019304E7019304
:1013F0000FE3019300E010E100938101109382015B
:10140000F3DEFF248395FDC153FF02C0577F8BE0BD
:10141000F8C1ECE9F0E000E2019300E2019300E2A0
:10142000019300E2019300E2019300E2019300E2E4
:1014300001930EE3019304E401930DE4019304E4AA
:10144000019300E2019304E4019309E601930DE6A0
:1014500001930FE3019300E010E1009381011093E9
:101460008201C2DEFF248395CCC153FF03C0577FA6
:1014700085E104C0C6C153FF19C0577F00918301A5
:101480000395083009F400270093830110E3100F3F
:10149000ECE9F0E0178718E8010F0BBB03E908BB84
:1014A000C4980000C49A08E000938101AAC188276B
:1014B00001E0F02EA6C1ECE9F0E000E2019300E2C9
:1014C000019300E2019300E2019300E2019300E244
:1014D000019300E201930EE301930CE4019305E410
:1014E000019304E4019300E2019304E4019309E60B
:1014F00001930DE601930FE3019300E010E10093E7
:1015000081011093820170DEFF2483957AC153FF1D
:1015100003C0577F8AE104C074C153FFDEC0577F08
:10152000009184010395053009F40027009384019C
:1015300010E3100FECE9F0E0178708E00093810159
:1015400000918401003039F5E5EEF0E000EF019301
:1015500008EF019300EE01930CED019300EF01936E
:1015600008EE019300EF019308EF019307E8019360
:1015700008EF019300EF019308EE019304ED01934E
:1015800008EF019300EE019308EF019300EF019340
:101590000FE80193A2C0013039F5E5EEF0E000EE6E
:1015A000019300EF019308EC019304EF019300EE27
:1015B00001930AE9019300EE019300EF01930DEC12
:1015C000019300EF019300EE01930AE9019304EE09
:1015D000019300EF019308EC019300EF019300EEFB
:1015E00001930FE9019379C0023039F5E5EEF0E09F
:1015F00000E0019300EC019300E2019308ED0193F8
:1016000000E0019304EE019300E1019300E80193EF
:101610000BE6019300E8019300E5019304EA0193CE
:1016200008E4019300E9019300E6019300E80193C7
:1016300000E001930FEF019350C0033039F5E5EE60
:10164000F0E000E0019300E0019300E8019300E77F
:10165000019300E001930CE8019300E4019300E0A2
:10166000019303EB019300E0019300E401930CE884
:10167000019300E3019300E4019300E8019300E08B
:10168000019300E001930FEF019327C0E5EEF0E036
:1016900000E0019300E0019300E0019300E001937A
:1016A00000E001930FEF019300E0019300E001934C
:1016B00000E0019300E0019300E001930FEF01933C
:1016C00000E0019300E0019300E0019300E001934A
:1016D00000E001930FEF019300C093C0882701E061
:1016E000F02E8FC0FF243092850140928601D8DC15
:1016F000839587C001E00BBB01E108BBC4980000E3
:10170000C49A53FF0BC0577F009185011AE0010F67
:101710000E3108F00E5100938501C2DC72C000E06A
:101720000BBB01E108BBC4980000C49A01E00BBBED
:1017300005E108BBC4980000C49A53FF0FC0577F4F
:10174000009185010395102F1A3010F01A50FCCF2C
:10175000103009F40A5000938501A2DC52C000E069
:101760000BBB05E108BBC4980000C49A01E00BBBA9
:101770000DE108BBC4980000C49A53FF0BC0577F0B
:10178000009186011AE0010F0C3308F00C5300930E
:10179000860186DC36C000E00BBB0DE108BBC498B7
:1017A0000000C49A01E00BBB01E308BBC498000031
:1017B000C49A53FF0FC0577F009186010395102FE5
:1017C0001A3010F01A50FCCF103009F40A50009370
:1017D000860166DC16C000E00BBB01E308BBC498C1
:1017E0000000C49A882700918501083108F008514B
:1017F000302E409086015524662701E0F02EAADAAB
:1018000000C00895E894BB275F9908C00091870144
:101810000030D1F3B017C0F3689408955C996894D0
:101820000CB10895E8945F9BFECF5C9968940CB16D
:1018300008955D9BFECF0CB908955F9B08955C9958
:1018400054C10CB1013009F41FC0033009F43BC08E
:10185000043009F46BC0053009F48BC0063009F47C
:10186000A1C0073009F4B0C0083009F4BFC002308D
:1018700009F4D9C0093009F4F3C00A3009F412C1DF
:101880000F3F09F422C126C1ACE3E7E3F1E0BADF80
:101890000EF42BC10F3F09F41DC10193AA95B9F7AE
:1018A000B1DF0EF422C10F3F09F014C11CE3A0E622
:1018B000B0E0E7E3F1E001910D931A95E1F705E55A
:1018C0000E94190C06C1E7E3F1E09CDF0EF40DC1A4
:1018D0000F3F09F4FFC0063408F0FCC0083008F4DC
:1018E000F9C00193A02F8EDF0EF4FFC00F3F09F463
:1018F000F1C00193AA95B9F785DF0EF4F6C00F3F4A
:1019000009F0E8C0E7E3F1E01191ACE9B0E0019142
:101910000D931A95E1F700E01091370100938101D2
:101920001093820105E50E94190CD3C06BDF0EF401
:10193000DCC0083008F0CEC0102F64DF0EF4D5C034
:101940000F3F09F0C7C01093830108E8010F0BBBDC
:1019500003E908BBC4980000C49A109181011030BB
:1019600019F01A951A951093810105E50E94190C3A
:10197000B0C0E7E3F1E0A8E045DF0EF4B6C00F3FEA
:1019800009F4A8C00193AA95B9F73CDF0EF4ADC0E5
:101990000F3F09F09FC0E7E3F1E073DC05E50E942B
:1019A000190C97C02FDF0EF4A0C0033008F092C0CE
:1019B000102F28DF0EF499C00F3F09F08BC0F12ED5
:1019C00005E50E94190C85C01DDF0EF48EC00A309B
:1019D00008F080C0102F16DF0EF487C00F3F09F00B
:1019E00079C0712F05E50E94190C73C0A2E1E7E3ED
:1019F000F1E008DF0EF479C00193AA95D1F702DF78
:101A00000EF473C00F3F09F065C012E1A5EEB0E01F
:101A1000E7E3F1E001910D931A95E1F705E50E94E6
:101A2000190C57C056C0EEDE0EF45FC00C3308F040
:101A300051C0102FE7DE0EF458C00F3F09F44AC022
:101A4000A02FE0DE0EF451C00F3F09F043C0E0E6E6
:101A5000F0E0E10FF11DA08305E50E94190C39C0EB
:101A6000D1DE0EF442C0083108F034C0102FCADEB7
:101A70000EF43BC00C3308F02DC0A02FC3DE0EF4D3
:101A800034C00C3308F026C0A02EBCDE0EF42DC0EE
:101A90000F3F09F01FC0312E4A2E5A2C05E50E9437
:101AA000190C17C0AFDE0EF420C00F3F09F412C0AE
:101AB000102FA8DE0EF419C00F3F09F00BC01093D1
:101AC000870105E50E94190C04C00FEF0E94190C54
:101AD00000C008950AEA0E94190CA4DE36F00F3FF8
:101AE000E1F70FEF0E94190CF4CF0EEE0E94190CD3
:101AF000F4CFE0E6F0E0ACE31192AA95E9F7E2EE6C
:101B0000F0E000E0019300E0019300E00193ECE9D4
:101B1000F0E000E2019300E2019300E2019300E2B1
:101B2000019300E2019300E2019300E2019300E2DD
:101B30000193E5EEF0E000EE019300EF019308EC75
:101B4000019304EB019300EE019308ED019300EE85
:101B5000019300EF01930FE8019300EF019300EE72
:101B6000019308ED019304EA019300EF019308EC5F
:101B7000019300EF019300EE01930FE90193E7EF6A
:101B8000F0E001E0019301E0019302E0019304E041
:101B9000019308E0019300E1019300E2019300E466
:101BA000019300E8019300E8019300E8019300E845
:101BB000019300E8019300E8019300E8019300E835
:101BC000019300E8019300E8019300E8019300E429
:101BD000019300E4019300E2019300E1019308E026
:101BE000019304E0019302E0019301E0019301E01D
:101BF000019301E0019301E0019301E0019301E011
:101C00000193E7E1F1E001E0019301E0019302E0DB
:101C1000019302E0019302E0019304E0019304E0E8
:101C2000019304E0019308E0019308E0019300E1CF
:101C3000019300E1019300E1019300E1019300E1D0
:101C4000019308E0019304E0019302E0019301E0B5
:101C5000019300E0019300E0019300E0019300E0B4
:101C6000019300E0019300E0019300E0019300E0A4
:101C7000019300E0019300E0019300E0019300E094
:101C8000019300E001930895ECE9F0E000E2019394
:101C900006E3019300E3019304E7019308E601934F
:101CA00000E201930CE6019305E701930DE6019331
:101CB00009E601930EE601930FE6019305E7019310
:101CC00003E7019300E2019303E401930CE4019321
:101CD0000FE401930CE401930BE4019300E2019300
:101CE00000E2019300E2019300E2019304E6019314
:101CF00005E6019303E7019309E6019307E60193E3
:101D00000EE6019305E6019304E6019300E20193D8
:101D10000DE2019300E2019300E201930DE40193CF
:101D20000DE2019304E5019305E6019303E60193B7
:101D300008E6019300E2019304E6019305E60193AE
:101D400003E7019309E6019307E601930EE6019389
:101D500000E2019309E401930EE6019303E6019387
:101D60000EE2019300E2019300E2019300E201938D
:101D700000E2019300E2019300E2019300E201938B
:101D800000E2019300E2019300E2019300E201937B
:101D900000E2019300E012E40093810110938201BC
:061DA00023DAFF24089580
:00000001FF
